:020000020000FC
:020000005EC0E0
:02001800BDC168
:02003C0023C2DD
:0200800088C234
:0200B4002AC35D
:1000BC00CFC201E20EBF0FEF0DBF07E104B908E09C
:1000CC0005B901E00DBD00E50CBD289A2C980F9ADE
:1000DC0017980000179A0CE000936A0000E20DBB21
:1000EC00259A269A2D982E982227992789E250E056
:1000FC0000E0A02EB02EA89500E004BF0EE1009306
:10010C00600000E0009360000BEA009364000FE3D2
:10011C000093650000E900BF00E20093B60006E022
:10012C000093B1000091B6000F71E1F707E007BB37
:10013C0001E00093700040E81CD1C6D003EC289875
:10014C0012D1002710D1289A00EE28980CD100EA81
:10015C000AD1289A01EE289806D10BE204D1289AEC
:10016C0002EE289800D103ECFED0289A03EE2898D2
:10017C00FAD004EAF8D0289A08EC2898F4D00BE2CC
:10018C00F2D0289A05EC2898EED000E8ECD0289A0A
:10019C000CEE2898E8D008E3E6D0289A0EEE2898C2
:1001AC00E2D005E0E0D0289A0DEE2898DCD000E0F3
:1001BC00DAD0289A0FE82898D6D0289A0EEC2898EE
:1001CC00D2D008E0D0D0289AA8950EE10093600018
:1001DC0008E2009360000FEF0CBB78942C9A07E0B8
:1001EC0003BF65E088950000000000006A95D1F718
:1001FC00002703BF2C9848E2BCD06CD0A5D030EAC5
:10020C004FEFB7D0863D39F13A95D1F76CD0E6CFA8
:10021C006AD063D100E00093A1000093720000004B
:10022C00000000005230D9F300E0009391000093DD
:10023C0021010093810000937100009373000093DF
:10024C0080000BEA009364000FE3009365002D9887
:10025C002E9850E0C3CF03EA0093640007E00093AC
:10026C00650003EA0093800000E00093890000938E
:10027C00880000938B0000938A000AE000938100B1
:10028C000FD10000000000005130D9F300E00093C2
:10029C00A5000093A40001E00093720002E000931B
:1002AC00A10058D20000000000008932D9F788273D
:1002BC000000000000008932D9F7882700000000F8
:1002CC0000008932D9F7A4CF02EC28984CD008E072
:1002DC004AD0289A01E8289846D000E044D0289AC1
:1002EC000830C1F7089502EC28983DD003E03BD0CC
:1002FC00289A000000000000000001E8289833D084
:10030C0000E031D0289A083071F7089502EC289853
:10031C002AD009E028D0289A01E8289824D000E0B7
:10032C0022D0289A0930C1F7089502EC28981BD0E6
:10033C0009E119D0289A01E8289815D000E013D0CB
:10034C00289A0931C1F7089502EC28980CD006E1DF
:10035C000AD0289A01E8289806D000E004D0289A00
:10036C000631C1F708950EBD0DB507FFFDCF0EB5D3
:10037C0008950000000000000000000000000000D4
:10038C0000004A95B1F708950F930FB70F930FE83C
:10039C002898E9DF289A01E82898E5DF00E0E3DFF8
:1003AC00289A063139F0013129F00F31A1F30231CD
:1003BC0091F336C0002400E22898D5DF00E0D3DFAB
:1003CC00003171F500E0CFDF00E0CDDF00E0CBDFE6
:1003DC00003059F1023021F500E0C5DF00E0C3DF49
:1003EC0000E0C1DF00E0BFDF00E0BDDF0031C1F4A1
:1003FC0000E0B9DF0B32A1F400E0B5DF002E00E025
:10040C00B2DF073669F400E0AEDF013C49F400E0EE
:10041C00AADF0A3829F400E0A6DF0F3909F4902985
:10042C00289A0F910FBF0F91189500E09CDF00E008
:10043C009ADF00E098DF00E096DF00E094DF0435FF
:10044C0079F700E090DF0B3B59F700E08CDF002ED2
:10045C0000E089DF0B3A21F700E085DF063401F775
:10046C0000E081DF0733E1F600E07DDF023DC1F6FD
:10047C00802DAA24BB24D4CF0000000000000F93D1
:10048C000FB70F9301E0A00E0027B01E28F0A8951F
:10049C000F910FBF0F911895000000000000FCCFCA
:1004AC0000E000939500009394000EE400939900F3
:1004BC0000E20093980002E00093710005E00093C5
:1004CC0091000FEF009389000093880000E00093E7
:1004DC008B0000938A0051E0089500E00093250101
:1004EC00009324010EE40093290100E200932801FB
:1004FC0002E00093730005E0009321010FEF0093DD
:10050C008B0000938A0000E0009389000093880020
:10051C0052E008955330B9F05430A9F000E0009344
:10052C0095000093940001E00093990000E0009383
:10053C00980002E0009371000AE000939100B0E291
:10054C00AA27D4E2CC2753E008955530D1F0563089
:10055C00C1F000E0009325010093240102E0009318
:10056C00290100E00093280102E0009373000AE0E7
:10057C00009321010FE300938B0000938A00D0E2DB
:10058C00CC2755E008950F930FB70F93513069F0B6
:10059C005330C9F05430B9F000E00093910000934F
:1005AC0071000F910FBF0F91189500E0009391000F
:1005BC0000937100009389000093880050E00F9124
:1005CC000FBF0F911895FE0105901590F772400121
:1005DC0003EBCDD0EF0190928B0080928A00FD014D
:1005EC0005901590400103EBC2D0DF01F83241F0C9
:1005FC0090928900809288000F910FBF0F911895EF
:10060C00543051F0B0E2AA27909289008092880071
:10061C000F910FBF0F91189500E00093910000937C
:10062C007100009389000093880000938B00009365
:10063C008A00042D013039F0033029F08BD00F9152
:10064C000FBF0F91189581DF0F910FBF0F91189568
:10065C000F930FB70F93523069F05530C9F05630E5
:10066C00B9F000E000932101009373000F910FBFCC
:10067C000F91189500E000932101009373000093F3
:10068C008B0000938A0050E00F910FBF0F911895CB
:10069C00FE0105901590400100E869D0EF01F83299
:1006AC0041F090928900809288000F910FBF0F91BA
:1006BC001895563051F0D0E2CC2790928900809258
:1006CC0088000F910FBF0F91189500E00093210146
:1006DC0000937300009389000093880000938B00B3
:1006EC0000938A00042D023029F034D00F910FBFF3
:1006FC000F9118950FDF0F910FBF0F9118950F9356
:10070C000FB70F93903061F0913099F09230B9F0AF
:10071C00933079F0492E99270F910FBF0F911895AF
:10072C00533019F0553019F0F5CF54E0F3CF56E0B3
:10073C00F1CF5330D1F35430C1F307DFEBCF553049
:10074C00B1F35630A1F3E6DEE5CF54E0E3CFE2DEC1
:10075C00FCDEE0CF02E0009389000CEC00938800F3
:10076C0000E000938B0000938A0057E00895909E60
:0E077C001001809E0027210C301E41010895BF
:1020000000000000000000000000000000000000D0
:1020100001000100010001000100020002000200B5
:102020000200030003000300040004000500050093
:102030000600060006000700080008000900090065
:102040000A000A000B000C000C000D000E000F002F
:102050000F001000110012001300130014001500EF
:1020600016001700180019001A001B001C001D00A4
:102070001E001F0020002100220023002500260052
:102080002700280029002B002C002D002E003000F6
:1020900031003200340035003700380039003B0091
:1020A0003C003E003F004100420044004600470023
:1020B00049004A004C004E004F00510053005400AC
:1020C000560058005A005B005D005F00610063002D
:1020D0006500660068006A006C006E0070007200A7
:1020E0007400760078007A007C007E008000820018
:1020F0008400860089008B008D008F009100930082
:10210000960098009A009C009F00A100A300A600E2
:10211000A800AA00AD00AF00B100B400B600B8003E
:10212000BB00BD00C000C200C500C700CA00CC0093
:10213000CF00D100D400D600D900DB00DE00E100E2
:10214000E300E600E800EB00EE00F000F300F6002C
:10215000F800FB00FE0000010301060109010B016C
:102160000E0111011401160119011C011F012201A8
:10217000250127012A012D013001330136013901E2
:102180003B013E014101440147014A014D0150011B
:102190005301560159015C015F016201650168014B
:1021A0006B016E017101740177017A017D0180017B
:1021B0008301860189018C018F01920195019801AB
:1021C0009B019E01A101A501A801AB01AE01B101D6
:1021D000B401B701BA01BD01C001C401C701CA0100
:1021E000CD01D001D301D601D901DD01E001E30128
:1021F000E601E901EC01EF01F201F601F901FC0150
:10220000FF010202050208020C020F02120215026F
:1022100018021B021E022102250228022B022E0296
:102220003102340237023A023E02410244024702BE
:102230004A024D0250025302560259025D026002E8
:102240006302660269026C026F0272027502780212
:102250007B027E028102840287028A028D02900242
:102260009302960299029C029F02A202A502A80272
:10227000AB02AE02B102B402B702BA02BD02C002A2
:10228000C302C502C802CB02CE02D102D402D702D9
:10229000D902DC02DF02E202E502E802EA02ED0214
:1022A000F002F302F502F802FB02FE020003030350
:1022B000060308030B030E0310031303160318038E
:1022C0001B031D0320032303250328032A032D03D7
:1022D0002F0332033403370339033C033E03410326
:1022E0004303460348034A034D034F03510354037A
:1022F000560358035B035D035F03620364036603D5
:1023000068036B036D036F03710373037503780335
:102310007A037C037E03800382038403860388039D
:102320008A038C038E03900392039403960398030D
:1023300099039B039D039F03A103A303A403A60387
:10234000A803AA03AB03AD03AF03B003B203B40306
:10235000B503B703B803BA03BC03BD03BF03C0038F
:10236000C203C303C503C603C703C903CA03CC031F
:10237000CD03CE03D003D103D203D303D503D603B9
:10238000D703D803D903DB03DC03DD03DE03DF035C
:10239000E003E103E203E303E403E503E603E70309
:1023A000E803E903EA03EB03EB03EC03ED03EE03BD
:1023B000EF03EF03F003F103F203F203F303F4037B
:1023C000F403F503F503F603F603F703F803F80344
:1023D000F803F903F903FA03FA03FB03FB03FB0316
:1023E000FC03FC03FC03FC03FD03FD03FD03FD03F1
:1023F000FD03FE03FE03FE03FE03FE03FE03FE03D6
:10240000FE03FE03FE03FE03FE03FE03FE03FE03C4
:10241000FD03FD03FD03FD03FD03FC03FC03FC03BF
:10242000FC03FB03FB03FB03FA03FA03F903F903C1
:10243000F803F803F803F703F603F603F503F503CF
:10244000F403F403F303F203F203F103F003EF03E5
:10245000EF03EE03ED03EC03EB03EB03EA03E90305
:10246000E803E703E603E503E403E303E203E10330
:10247000E003DF03DE03DD03DC03DB03D903D80362
:10248000D703D603D503D303D203D103D003CE039E
:10249000CD03CC03CA03C903C703C603C503C303E3
:1024A000C203C003BF03BD03BC03BA03B803B70331
:1024B000B503B403B203B003AF03AD03AB03AA0388
:1024C000A803A603A403A303A1039F039D039B03E7
:1024D0009903980396039403920390038E038C034D
:1024E0008A03880386038403820380037E037C03BC
:1024F0007A0378037503730371036F036D036B0332
:1025000068036603640362035F035D035B035803B0
:102510005603540351034F034D034A034803460334
:10252000430341033E033C033903370334033203BF
:102530002F032D032A0328032503230320031D0350
:102540001B0318031603130310030E030B030803E6
:10255000060303030003FE02FB02F802F502F30286
:10256000F002ED02EA02E802E502E202DF02DC022A
:10257000D902D702D402D102CE02CB02C802C502D0
:10258000C302C002BD02BA02B702B402B102AE0277
:10259000AB02A802A502A2029F029C029902960227
:1025A000930290028D028A028702840281027E02D7
:1025B0007B027802750272026F026C026902660287
:1025C000630260025D0259025602530250024D023C
:1025D0004A024702440241023E023A0237023402F2
:1025E00031022E022B022802250221021E021B02AA
:1025F0001802150212020F020C0208020502020262
:10260000FF01FC01F901F601F201EF01EC01E90122
:10261000E601E301E001DD01D901D601D301D001DA
:10262000CD01CA01C701C401C001BD01BA01B70192
:10263000B401B101AE01AB01A801A501A1019E0148
:102640009B019801950192018F018C0189018601FE
:10265000830180017D017A017701740171016E01AE
:102660006B016801650162015F015C01590156015E
:10267000530150014D014A014701440141013E010E
:102680003B0139013601330130012D012A012701B7
:10269000250122011F011C0119011601140111015C
:1026A0000E010B010901060103010001FE00FB0000
:1026B000F800F600F300F000EE00EB00E800E600A2
:1026C000E300E000DE00DB00D900D600D400D1003A
:1026D000CF00CC00CA00C700C500C200C000BD00CA
:1026E000BB00B800B600B400B100AF00AD00AA0056
:1026F000A800A600A300A1009F009C009A009800DB
:102700009600930091008F008D008B008900860059
:102710008400820080007E007C007A0078007600D1
:102720007400720070006E006C006A006800660041
:102730006500630061005F005D005B005A005800A7
:1027400056005400530051004F004E004C004A0008
:102750004900470046004400420041003F003E005F
:102760003C003B00390038003700350034003200AF
:10277000310030002E002D002C002B0029002800F5
:1027800027002600250023002200210020001F0032
:102790001E001D001C001B001A0019001800170065
:1027A0001600150014001300130012001100100091
:1027B0000F000F000E000D000C000C000B000A00B3
:1027C0000A000900090008000800070006000600CA
:1027D00006000500050004000400030003000300D8
:1027E00002000200020002000100010001000100DD
:1027F00001000000000000000000000000000000D8
:00000001FF
